:020000040000FA
:0A0000000000000093EF00F0A3D011
:08001800F6D09EA8FED7AD6EE4
:100020001200146E960E0B6E980E0C6E55D8D8B446
:10003000CA90D8A4CA80FC0FD8A0CA92D8B0CA82ED
:10004000800E0B6E960E0C6E980E0F6E106ACAB074
:1000500025D8CAB223D842D80B04CB6E0BC00DF002
:100060000CC00EF00250116E126E023C126A4BD898
:100070001050142E0AD0BE6E0C0EBD6E0FBEBD8A7F
:100080000FBCBD889494CA841200BB6E0C0EBA6E6D
:100090000FBEBA8A0FBCBA889492F5D700D8D89010
:1000A0000F320C320B3212000E6A0D6EFF0E0D264F
:1000B0000E2200D0D8A01200030E0C6EE60E02D85D
:1000C000F5D70C6AFE0F0B6EE86A0C5AD8A0120026
:1000D00000000B0600D0F8D7106A0F6A100EF36EFE
:1000E0000C340F3610360D500F5C0E50105805E3CF
:1000F0000D500F5E0E50105AD8800B360C36F32E72
:10010000EFD70B5012000D501102F3CF0FF0F4CFC8
:1001100010F00E501102F35010260D501202F35041
:1001200010260F501200006AB8964F0EAF6EB06ADC
:10013000240EAC6E900EAB6E00010F0EC16E070E5A
:10014000B46EC69A400E926E936AC00E946E35D10C
:10015000F2A409D0F2941E4A1F2AD6CF1CF0D7CFA2
:100160001DF0827011009EAA19D0060EAB1412E188
:10017000E2CF34F0E1CF33F0352A10EE3CF03550C9
:10018000E126000EE222AECFE7FF34C0E2FF33C02B
:10019000E1FF1100AE50AE50AB98AB881100355066
:1001A000365C14E0362AEACF0CF0E9CF0BF000EE13
:1001B0003CF03650E926000EEA22EF50326E0CC0B9
:1001C000EAFF0BC0E9FFD880120004D0E868326E65
:1001D000D8A012001200356A366A9D8A9F8AF28E74
:1001E000F28C12009D9A00EE3CF0010EF46EF36A60
:1001F000F306000EF45AEE6AF450F310F9E1356A92
:10020000366A9D8A1200F29EE0CF7FF4EACF80F436
:10021000E9CF81F402C082F40BC083F40CC084F4F3
:100220000DC085F40EC086F40FC087F410C088F4AA
:1002300011C089F412C08AF413C08BF414C08CF47A
:1002400015C08DF416C08EF417C08FF418C090F44A
:1002500019C091F41AC092F41BC093F4F4CF94F433
:10026000F3CF95F4D8CF96F4E8CF97F4F28E00014F
:10027000A192010162510001E8A06AD0196A7CC113
:1002800018F00F0E1816000E19161B6A7EC11AF010
:100290000F0E1A16000E1B161A5018121B501912A8
:1002A0001B6A7DC11AF00F0E1A16000E1B1618508D
:1002B0001A10376E196A7CC118F0F00E1816000E6D
:1002C00019161B6A7EC11AF0F00E1A16000E1B16C4
:1002D0001A5018121B5019121B6A7DC11AF0F00E29
:1002E0001A16000E1B1618501A10386E38380F0BDD
:1002F000386E37520BE0C00E026E4C0E0E6E500E72
:100300000D6E010E8EDE010E396E08D0026A4C0EA3
:100310000E6E500E0D6E010E84DE396A38520AE000
:10032000C00E026E4C0E0E6E500E0D6E020E79DE79
:10033000392A08D0026A4C0E0E6E500E0D6E020E57
:1003400070DE396A020E395C02E18B8601D08B9631
:10035000F29E7FC4E0FF80C4EAFF81C4E9FF82C44B
:1003600002F083C40BF084C40CF085C40DF086C485
:100370000EF087C40FF088C410F089C411F08AC44D
:1003800012F08BC413F08CC414F08DC415F08EC41D
:1003900016F08FC417F090C418F091C419F092C4ED
:1003A0001AF093C41BF094C4F4FF95C4F3FF96C4F1
:1003B000D8FF97C4E8FFF28E100094908B90010153
:1003C000616B000194908B80C80E6EDE94908B90D0
:1003D000939E8A9E939C8A9C9290899092928992F5
:1003E000939A8A9A93988A989294899492968996E5
:1003F00093968A9693948A9492988998929A899AD5
:1004000093928A9293908A90949A8B9A94988B98CC
:100410002E6801EE40F0200EEE68E82EFDD7026A4D
:100420004C0E0E6E500E0D6E020E11EC00F0026AB4
:100430004C0E0E6E500E0D6E010E11EC00F09496E7
:100440008B968BEC0CF02E6801EE40F0200EEE68DF
:10045000E82EFDD701017C6B7E6B7D6B7B6B6B6B3C
:100460006C6B6D6B6E6B6F6B706B716B726B736BB8
:10047000746B756B766B776B786B796B7A6B636B80
:10048000646B656B666B676B686B696B6A6B6281CB
:10049000A2DE0001A7DECD6AF294F28A870ED56E45
:1004A000B16AA192A082B36AB26AD08EA292B10E52
:1004B000B16EB70E0DEC00F0420E0DEC00F0000E28
:1004C0000DEC00F0D6CF1CF0D7CF1DF068DE32C0A7
:1004D00020F0B80E205C09E3FE0E205C03E353EF2E
:1004E00006F003D0216A53EF06F020AE38D0216A1F
:1004F000870E205C05E120C021F0226823682DD002
:10050000970E205C05E120C021F02468256825D0E5
:10051000A70E205C05E120C021F0266827681DD0C9
:10052000B70E205C05E120C021F02868296815D0AD
:10053000C70E205C04E120C021F02A680ED0D70E3F
:10054000205C04E120C021F02B6807D0E70E205C7E
:1005500004E120C021F02C682D684DEF06F02152F7
:1005600004E153EF06F04DEF06F0870E215CD8A4AE
:1005700076D0222803E120C022F06FD020C023F0E3
:10058000410E225C07E189900101636B7B917D91B3
:10059000000162D0430E225C07E189920101646B85
:1005A0007B937D93000158D0450E225C07E189942E
:1005B0000101656B7B957D9500014ED0480E225C54
:1005C00007E189960101666B7B977D97000144D016
:1005D0004A0E225C07E189980101676B7B997D993E
:1005E00000013AD04D0E225C07E1899A0101686B47
:1005F0007B9B7D9B000130D04F0E225C07E18B9AE4
:100600000101696B7B9D7D9D000126D0510E225C0E
:1006100007E18B9801016A6B7B9F7D9F00011CD0D5
:10062000780E225C09E1026A4C0E0E6E500E0D6EC1
:10063000010E11EC00F010D0790E225C09E1026A83
:100640004C0E0E6E500E0D6E020E11EC00F004D02A
:100650007A0E225C01E18B9622684DEF06F0970E30
:10066000215CD8A4B5EF05F0242804E120C024F0D3
:10067000B4EF05F020C025F02552D8A46ED0410E6D
:10068000245C07E189900101636B7B917D910001FE
:1006900062D0430E245C07E189920101646B7B9375
:1006A0007D93000158D0450E245C07E18994010137
:1006B000656B7B957D9500014ED0480E245C07E16B
:1006C00089960101666B7B977D97000144D04A0EA5
:1006D000245C07E189980101676B7B997D99000192
:1006E0003AD04D0E245C07E1899A0101686B7B9B2F
:1006F0007D9B000130D04F0E245C07E18B9A0101F5
:10070000696B7B9D7D9D000126D0510E245C07E125
:100710008B9801016A6B7B9F7D9F00011CD0780E36
:10072000245C09E1026A4C0E0E6E500E0D6E010E35
:1007300011EC00F010D0790E245C09E1026A4C0E35
:100740000E6E500E0D6E020E11EC00F004D07A0EFB
:10075000245C01E18B96B3EF05F0410E245C38E197
:1007600001017E31000133E225C063F103EE7FF029
:10077000D89001016335E926000EEA22EECF07F09A
:10078000EFCF08F007501C24036E08501D20046EA4
:10079000000E1E20056E000E1F20066E03C040F1E5
:1007A00004C041F105C042F106C043F189807C815B
:1007B0007E81608163C16BF17D917353000104E020
:1007C00001017B81000102D001017B910001CBD1AD
:1007D000430E245C39E101017E510001E8B233D0BF
:1007E00025C064F103EE7FF0D89001016435E9265D
:1007F000000EEA22EECF07F0EFCF08F007501C24DE
:10080000036E08501D20046E000E1E20056E000EA3
:100810001F20066E03C044F104C045F105C046F137
:1008200006C047F189827C837E83608164C16CF15C
:100830007D937453000104E001017B83000102D029
:1008400001017B9300018FD1450E245C39E1010148
:100850007E510001E8B433D025C065F103EE7FF08E
:10086000D89001016535E926000EEA22EECF07F0A7
:10087000EFCF08F007501C24036E08501D20046EB3
:10088000000E1E20056E000E1F20066E03C048F1EC
:1008900004C049F105C04AF106C04BF189847C854A
:1008A0007E85608165C16DF17D957553000104E021
:1008B00001017B85000102D001017B95000153D12C
:1008C000480E245C39E101017E510001E8B633D0C5
:1008D00025C066F103EE7FF0D89001016635E92668
:1008E000000EEA22EECF07F0EFCF08F007501C24ED
:1008F000036E08501D20046E000E1E20056E000EB3
:100900001F20066E03C04CF104C04DF105C04EF12E
:1009100006C04FF189867C877E87608166C16EF153
:100920007D977653000104E001017B87000102D02E
:1009300001017B97000117D14A0E245C39E10101C6
:100940007E510001E8B833D025C067F103EE7FF097
:10095000D89001016735E926000EEA22EECF07F0B4
:10096000EFCF08F007501C24036E08501D20046EC2
:10097000000E1E20056E000E1F20066E03C050F1F3
:1009800004C051F105C052F106C053F189887C8939
:100990007E89608167C16FF17D997753000104E022
:1009A00001017B89000102D001017B990001DBD0AC
:1009B0004D0E245C39E101017E510001E8BA33D0CB
:1009C00025C068F103EE7FF0D89001016835E92673
:1009D000000EEA22EECF07F0EFCF08F007501C24FC
:1009E000036E08501D20046E000E1E20056E000EC2
:1009F0001F20066E03C054F104C055F105C056F126
:100A000006C057F1898A7C8B7E8B608168C170F14A
:100A10007D9B7853000104E001017B8B000102D033
:100A200001017B9B00019FD04F0E245C39E1010145
:100A30007E510001E8BC33D025C069F103EE7FF0A0
:100A4000D89001016935E926000EEA22EECF07F0C1
:100A5000EFCF08F007501C24036E08501D20046ED1
:100A6000000E1E20056E000E1F20066E03C058F1FA
:100A700004C059F105C05AF106C05BF18B8A7C8D28
:100A80007E8D608169C171F17D9D7953000104E023
:100A900001017B8D000102D001017B9D000163D02B
:100AA000510E245C38E101017E35000133E225C09E
:100AB0006AF103EE7FF0D89001016A35E926000E55
:100AC000EA22EECF07F0EFCF08F007501C24036EA8
:100AD00008501D20046E000E1E20056E000E1F2003
:100AE000066E03C05CF104C05DF105C05EF106C096
:100AF0005FF18B887C8F7E8F60816AC172F17D9FF0
:100B00007A53000104E001017B8F000102D0010152
:100B10007B9F000128D0780E245C0FE1D89025300F
:100B20003A6E25503A263AC002F04C0E0E6E500E28
:100B30000D6E010E11EC00F016D0790E245C0FE161
:100B4000D89025303A6E25503A263AC002F04C0E25
:100B50000E6E500E0D6E020E11EC00F004D07A0EE7
:100B6000245C01E18B86246898D0A70E215C0BE100
:100B7000262803E120C026F005D020C027F0F5ECA0
:100B80000BF026688AD0B70E215CD8A472D0282832
:100B900003E120C028F06CD020C029F01E0E285C94
:100BA00016E129C073F129C074F129C075F129C07B
:100BB00076F129C077F129C078F129C079F129C0EF
:100BC0007AF1295202E101017B6B000150D0420E03
:100BD000285C17E1295209E101016191000154ECFF
:100BE0000CF001017B6B00010AD0010161818A8E4A
:100BF0008A8C8A8A8A888A868A848A828A80000184
:100C000036D0450E285C0AE1295204E101016291C7
:100C1000000102D001016281000129D07B0E285C15
:100C200025E189908992899489968998899A8B9AE5
:100C30008B98026A4C0E0E6E500E0D6E010E11EC6A
:100C400000F0026A4C0E0E6E500E0D6E020E11EC8C
:100C500000F08B9601EE40F0200EEE68E82EFDD7F6
:100C600001017C6B7E6B7D6B60817B6B0001286872
:100C700014D0C70E215C06E12A2802E120C02AF028
:100C80002A680BD0E70E215C08E12C2803E120C084
:100C90002CF003D020C02DF02C6801016031000140
:100CA00002E3B4EC0BF0080E2E5CD8B0A6EF0BF00C
:100CB00001013C511C5C3D511D583E511E583F5195
:100CC0001F580001D8A0A5EF0BF001013F8F2E5255
:100CD0000001D8A4A2D001017C31000126E3899053
:100CE00001017E8101EE7FF0D8906B35E926000E80
:100CF000EA22EECF07F0EFCF08F007501C24036E76
:100D000008501D20046E000E1E20056E000E1F20D0
:100D1000066E03C040F104C041F105C042F106C0B7
:100D200043F17C910001A4EF0BF001017E31000141
:100D300014E301017C9189907E917D914369426920
:100D4000416940697353000102E101017B91010196
:100D50007B310001D8A0A4EF0BF001017D3100012F
:100D600026E2899002EE7FF0D89001017335E926E2
:100D7000000EEA22EECF07F0EFCF08F007501C2458
:100D8000036E08501D20046E000E1E20056E000E1E
:100D90001F20066E03C040F104C041F105C042F1BE
:100DA00006C043F17D817E917C91000134D0010128
:100DB0007B31000126E301017C8103EE7FF0D890B6
:100DC0006335E926000EEA22EECF07F0EFCF08F0F8
:100DD00007501C24036E08501D20046E000E1E20B8
:100DE000056E000E1F20066E03C040F104C041F1E5
:100DF00005C042F106C043F189807E817D910001EA
:100E000009D0899001017C917D917E91436942696D
:100E1000416940690001A4EF0BF0010E2E5CD8A4DB
:100E2000A6D001017C510001E8A226D089920101DF
:100E30007E8301EE7FF0D8906C35E926000EEA2221
:100E4000EECF07F0EFCF08F007501C24036E0850D8
:100E50001D20046E000E1E20056E000E1F20066E63
:100E600003C044F104C045F105C046F106C047F196
:100E70007C930001A4EF0BF001017E510001E8A278
:100E800014D0899201017C937E937D9347694669D2
:100E9000456944697453000102E101017B9301013A
:100EA0007B510001E8A2A4EF0BF001017D5100018C
:100EB000E8B226D0899202EE7FF0D8900101743515
:100EC000E926000EEA22EECF07F0EFCF08F0075038
:100ED0001C24036E08501D20046E000E1E20056E9B
:100EE000000E1F20066E03C044F104C045F105C08A
:100EF00046F106C047F17D837E937C93000135D097
:100F000001017B510001E8A226D001017C8303EEA0
:100F10007FF0D8906435E926000EEA22EECF07F084
:100F2000EFCF08F007501C24036E08501D20046EFC
:100F3000000E1E20056E000E1F20066E03C044F139
:100F400004C045F105C046F106C047F189827E83A1
:100F50007D93000109D0899201017C937D937E935A
:100F600047694669456944690001A4EF0BF0020E28
:100F70002E5CD8A4A6D001017C510001E8A426D0A3
:100F8000899401017E8501EE7FF0D8906D35E926C8
:100F9000000EEA22EECF07F0EFCF08F007501C2436
:100FA000036E08501D20046E000E1E20056E000EFC
:100FB0001F20066E03C048F104C049F105C04AF184
:100FC00006C04BF17C950001A4EF0BF001017E51AE
:100FD0000001E8A414D0899401017C957E957D954B
:100FE0004B694A69496948697553000102E1010189
:100FF0007B9501017B510001E8A4A4EF0BF00101F6
:101000007D510001E8B426D0899402EE7FF0D8909B
:1010100001017535E926000EEA22EECF07F0EFCF89
:1010200008F007501C24036E08501D20046E000EAB
:101030001E20056E000E1F20066E03C048F104C07E
:1010400049F105C04AF106C04BF17D857E957C953E
:10105000000135D001017B510001E8A426D0010137
:101060007C8503EE7FF0D8906535E926000EEA22F4
:10107000EECF07F0EFCF08F007501C24036E0850A6
:101080001D20046E000E1E20056E000E1F20066E31
:1010900003C048F104C049F105C04AF106C04BF154
:1010A00089847E857D95000109D0899401017C9514
:1010B0007D957E954B694A69496948690001A4EFAD
:1010C0000BF0030E2E5CD8A4A6D001017C510001C8
:1010D000E8A626D0899601017E8701EE7FF0D890A0
:1010E0006E35E926000EEA22EECF07F0EFCF08F0CA
:1010F00007501C24036E08501D20046E000E1E2095
:10110000056E000E1F20066E03C04CF104C04DF1A9
:1011100005C04EF106C04FF17C970001A4EF0BF023
:1011200001017E510001E8A614D0899601017C9747
:101130007E977D974F694E694D694C6976530001E2
:1011400002E101017B9701017B510001E8A6A4EFB8
:101150000BF001017D510001E8B626D0899602EE20
:101160007FF0D89001017635E926000EEA22EECF15
:1011700007F0EFCF08F007501C24036E08501D2025
:10118000046E000E1E20056E000E1F20066E03C0AA
:101190004CF104C04DF105C04EF106C04FF17D8702
:1011A0007E977C97000135D001017B510001E8A6B4
:1011B00026D001017C8703EE7FF0D8906635E926C2
:1011C000000EEA22EECF07F0EFCF08F007501C2404
:1011D000036E08501D20046E000E1E20056E000ECA
:1011E0001F20066E03C04CF104C04DF105C04EF146
:1011F00006C04FF189867E877D97000109D08996C8
:1012000001017C977D977E974F694E694D694C69C6
:101210000001A4EF0BF0040E2E5CD8A4A5D00101B0
:101220007C510001E8A826D0899801017E8901EE51
:101230007FF0D8906F35E926000EEA22EECF07F056
:10124000EFCF08F007501C24036E08501D20046ED9
:10125000000E1E20056E000E1F20066E03C050F10A
:1012600004C051F105C052F106C053F17C99000150
:10127000A4EF0BF001017E510001E8A814D0899879
:1012800001017C997E997D99536952695169506930
:101290007753000102E101017B9901017B510001BB
:1012A000E8A8A4EF0BF001017D510001E8B826D0B9
:1012B000899802EE7FF0D89001017735E926000E7B
:1012C000EA22EECF07F0EFCF08F007501C24036EA0
:1012D00008501D20046E000E1E20056E000E1F20FB
:1012E000066E03C050F104C051F105C052F106C0B2
:1012F00053F17D897E997C99000135D001017B51A4
:101300000001E8A826D001017C8903EE7FF0D89087
:101310006735E926000EEA22EECF07F0EFCF08F09E
:1013200007501C24036E08501D20046E000E1E2062
:10133000056E000E1F20066E03C050F104C051F16F
:1013400005C052F106C053F189887E897D9900015C
:1013500009D0899801017C997D997E9953695269D8
:10136000516950690001F0D1050E2E5CD8A4A3D0BC
:1013700001017C510001E8AA25D0899A01017E8BE8
:1013800001EE7FF0D8907035E926000EEA22EECF0C
:1013900007F0EFCF08F007501C24036E08501D2003
:1013A000046E000E1E20056E000E1F20066E03C088
:1013B00054F104C055F105C056F106C057F17C9BAD
:1013C0000001C2D101017E510001E8AA13D0899A1F
:1013D00001017C9B7E9B7D9B5769566955695469C9
:1013E0007853000102E101017B9B01017B51000167
:1013F000E8AAAAD101017D510001E8BA26D0899A54
:1014000002EE7FF0D89001017835E926000EEA223D
:10141000EECF07F0EFCF08F007501C24036E085002
:101420001D20046E000E1E20056E000E1F20066E8D
:1014300003C054F104C055F105C056F106C057F180
:101440007D8B7E9B7C9B000135D001017B5100018F
:10145000E8AA26D001017C8B03EE7FF0D890683596
:10146000E926000EEA22EECF07F0EFCF08F0075092
:101470001C24036E08501D20046E000E1E20056EF5
:10148000000E1F20066E03C054F104C055F105C0C4
:1014900056F106C057F1898A7E8B7D9B000109D0E9
:1014A000899A01017C9B7D9B7E9B57695669556992
:1014B0005469000149D1060E2E5CD8A4A3D00101C5
:1014C0007C510001E8AC25D08B9A01017E8D01EEA4
:1014D0007FF0D8907135E926000EEA22EECF07F0B2
:1014E000EFCF08F007501C24036E08501D20046E37
:1014F000000E1E20056E000E1F20066E03C058F160
:1015000004C059F105C05AF106C05BF17C9D000191
:101510001BD101017E510001E8AC13D08B9A01016F
:101520007C9D7E9D7D9D5B695A6959695869795397
:10153000000102E101017B9D01017B510001E8AC4A
:1015400003D101017D510001E8BC26D08B9A02EE47
:101550007FF0D89001017935E926000EEA22EECF1E
:1015600007F0EFCF08F007501C24036E08501D2031
:10157000046E000E1E20056E000E1F20066E03C0B6
:1015800058F104C059F105C05AF106C05BF17D8DD8
:101590007E9D7C9D000135D001017B510001E8ACAE
:1015A00026D001017C8D03EE7FF0D8906935E926C5
:1015B000000EEA22EECF07F0EFCF08F007501C2410
:1015C000036E08501D20046E000E1E20056E000ED6
:1015D0001F20066E03C058F104C059F105C05AF12E
:1015E00006C05BF18B8A7E8D7D9D000109D08B9AB0
:1015F00001017C9D7D9D7E9D5B695A695969586991
:101600000001A2D0070E2E5CD8A49ED001017C352B
:10161000000125E38B9801017E8F01EE7FF0D890C9
:101620007235E926000EEA22EECF07F0EFCF08F080
:1016300007501C24036E08501D20046E000E1E204F
:10164000056E000E1F20066E03C05CF104C05DF144
:1016500005C05EF106C05FF17C9F000175D00101FD
:101660007E35000113E38B9801017C9F7E9F7D9F57
:101670005F695E695D695C697A53000102E101019D
:101680007B9F01017B350001D8A05ED001017D3533
:10169000000126E28B9802EE7FF0D89001017A35A6
:1016A000E926000EEA22EECF07F0EFCF08F0075050
:1016B0001C24036E08501D20046E000E1E20056EB3
:1016C000000E1F20066E03C05CF104C05DF105C072
:1016D0005EF106C05FF17D8F7E9F7C9F000134D05C
:1016E00001017B35000126E301017C8F03EE7FF0D1
:1016F000D8906A35E926000EEA22EECF07F0EFCF48
:1017000008F007501C24036E08501D20046E000EC4
:101710001E20056E000E1F20066E03C05CF104C083
:101720005DF105C05EF106C05FF18B887E8F7D9F05
:10173000000109D08B9801017C9F7D9F7E9F5F698E
:101740005E695D695C6900010FD80CD01FAC0AD0DE
:101750001F6A1E6A1D6A1C6A01EE40F0200EEE68C8
:10176000E82EFDD762EF02F02E6801013F8F3A6A42
:101770000001080E3A5C35E2D8903A34E96EEA6A24
:10178000EA36E936EA36400EE926010EEA22EFCFC4
:1017900003F0ECCF04F0ECCF05F0ECCF06F0010144
:1017A0003C51035C3D5104583E5105583F51065889
:1017B000000115E2D8903A34E96EEA6AEA36E93671
:1017C000EA36400EE926010EEA22EFCF3CF1ECCFDB
:1017D0003DF1ECCF3EF1ECCF3FF13AC02EF03A2A8A
:1017E000C7E30101609100011200410E265C08E18F
:1017F00027C073F1275202E101017B9100014CD017
:10180000430E265C08E127C074F1275202E1010172
:101810007B93000141D0450E265C08E127C075F19D
:10182000275202E101017B95000136D0480E265C6B
:1018300008E127C076F1275202E101017B97000100
:101840002BD04A0E265C08E127C077F1275202E12F
:1018500001017B99000120D04D0E265C08E127C0D4
:1018600078F1275202E101017B9B000115D04F0E58
:10187000265C08E127C079F1275202E101017B9D36
:1018800000010AD0510E265C07E127C07AF12752E9
:1018900002E101017B9F0001266812002A68120004
:1018A0002C6812002B6812008A9E8A9C8A9A8A9859
:1018B0008A968A948A928A90899089928994899644
:1018C0008998899A8B9A8B98026A4C0E0E6E500EEC
:1018D0000D6E010E11EC00F0026A4C0E0E6E500EF1
:1018E0000D6E020E11EC00F08B9601EE40F0200E12
:1018F000EE68E82EFDD701017C6B7E6B7D6B7B6B08
:10190000736B746B756B766B776B786B796B7A6BCB
:10191000608100011200020180697F69A20E826F5E
:10192000C30E816F020E3A6E0001800E3A5C20E217
:101930003A04096E02EE7FF0D8900934E926000ED1
:10194000EA22EECF07F0EFCF08F0330E075C036E0C
:10195000010E0858046E02EE7FF0D8903A34E92662
:10196000000EEA2203C0EEFF04C0EFFF3A2ADCE3D8
:101970000301826B7C0E816F0101826BF80E816F17
:10198000020E3A6E0001800E3A5CD8B048D03A049C
:10199000096E03EE7FF0D8900934E926000EEA22A2
:1019A000EECF07F0EFCF08F0020E0724036E000E13
:1019B0000820046E03EE7FF0D8903A34E926000E3A
:1019C000EA2203C0EEFF04C0EFFF03EE7FF0D890E1
:1019D0003A34E926000EEA22EECF07F0EFCF08F006
:1019E00003EE7FF0D8903A34E926000EEA22EECFDB
:1019F00009F0EFCF0AF009500724036E0A500820BF
:101A0000046E01EE7FF0D8903A34E926000EEA2207
:101A100003C0EEFF04C0EFFF3A2AD8A0B3D71200EC
:021A2000FFD7EE
:020000040030CA
:0300010006160ED2
:020005008580F4
:060008000FC00FE00F40E5
:00000001FF
